Microchip MPLAB XC8 Compiler V2.36

Linker command line:

-W-3 --edf=/opt/microchip/xc8/v2.36/pic/dat/en_msgs.txt -cn \
  -h+dist/default/production/UART_TX_18F452_2.X__copia_.production.sym \
  --cmf=dist/default/production/UART_TX_18F452_2.X__copia_.production.cmf \
  -z -Q18F452 -o/tmp/xcXPOGpBB --defsym=__MPLAB_BUILD=1 \
  -Mdist/default/production/UART_TX_18F452_2.X__copia_.production.map \
  --md=/tmp/xcXpKbmao.dat -E1 -ver=XC8 Compiler --acfsm=1493 \
  -ACODE=00h-03FFFhx2 -ACONST=00h-07FFFh -ASMALLCONST=0600h-06FFhx122 \
  -AMEDIUMCONST=0600h-07FFFh -ACOMRAM=01h-07Fh -AABS1=00h-05FFh \
  -ABIGRAM=01h-05FFh -ARAM=080h-0FFh,0100h-01FFhx5 -ABANK0=080h-0FFh \
  -ABANK1=0100h-01FFh -ABANK2=0200h-02FFh -ABANK3=0300h-03FFh \
  -ABANK4=0400h-04FFh -ABANK5=0500h-05FFh -ASFR=0F80h-0FFFh \
  -ABIGSFR=0F80h-0FFFh -ACONFIG=0300000h-030000Dh -AIDLOC=0200000h-0200007h \
  -AEEDATA=0F00000h-0F000FFh -peeprom_data=EEDATA \
  -preset_vec=00h,intcode=08h,intcodelo,powerup,init -pramtop=0600h \
  -psmallconst=SMALLCONST -pmediumconst=MEDIUMCONST -pconst=CONST \
  -AFARRAM=00h-00h \
  -prdata=COMRAM,nvrram=COMRAM,nvbit=COMRAM,rbss=COMRAM,rbit=COMRAM \
  -pfarbss=FARRAM,fardata=FARRAM,nvFARRAM=FARRAM \
  -pintsave_regs=BIGRAM,bigbss=BIGRAM,bigdata=BIGRAM -pbss=RAM \
  -pidata=CODE,irdata=CODE,ibigdata=CODE,ifardata=CODE -prparam=COMRAM \
  /tmp/xcXMhfnii.o \
  dist/default/production/UART_TX_18F452_2.X__copia_.production.o 

Object code version is 3.11

Machine type is 18F452



                Name                               Link     Load   Length Selector   Space Scale
/tmp/xcXMhfnii.o
                idloc                            200000   200000        8        0       5
                config                           300000   300000        E        0       4
                text                               1F70     1F70        2      FB8       0
                init                                 B2       B2        4        4       0
                reset_vec                             0        0        6        0       0
dist/default/production/UART_TX_18F452_2.X__copia_.production.o
                intcode                               8        8       AA        4       0
                idloc                            200000   200000        8        0       5
                config                           300000   300000        E        0       4
                temp                                 6F       6F        1        1       1
                smallconst                          600      600        A      300       0
                text31                             1DA2     1DA2       48      305       0
                text29                             1DEA     1DEA       34      305       0
                text28                             1F14     1F14        C      305       0
                text27                             1F08     1F08        C      305       0
                text26                             1E1E     1E1E       26      305       0
                text25                             1EA4     1EA4       1E      305       0
                text24                             1E44     1E44       24      305       0
                text23                             1E86     1E86       1E      305       0
                text22                             1A4C     1A4C       FA      305       0
                text21                             1C0C     1C0C       7C      305       0
                text20                             1E68     1E68       1E      305       0
                text19                             1C88     1C88       66      305       0
                text18                             1F52     1F52        A      305       0
                text17                             1F48     1F48        A      305       0
                text16                             1F3E     1F3E        A      305       0
                text15                             1F34     1F34        A      305       0
                text14                             1EDE     1EDE       1A      305       0
                text13                              60A      60A      5A8      305       0
                text12                             1056     1056      432      305       0
                text11                              BB2      BB2      4A4      305       0
                text10                             1916     1916      136      305       0
                text9                              1B46     1B46       C6      305       0
                text8                              1EF8     1EF8       10      305       0
                text7                              1F64     1F64        8      305       0
                text6                              1F5C     1F5C        8      305       0
                text5                              1EC2     1EC2       1C      305       0
                text4                              1D52     1D52       50      305       0
                text3                              1488     1488      358      305       0
                text2                              1F2A     1F2A        A      305       0
                text1                              1F20     1F20        A      305       0
                text0                              17E0     17E0      136      305       0
                cstackCOMRAM                          1        1       60        1       1
                cstackBANK0                          AA       AA       1A       80       1
                bssBANK2                            200      200       FF      200       1
                bssBANK1                            100      100       64      100       1
                bssBANK0                             80       80       2A       80       1
                dataCOMRAM                           6C       6C        3        1       1
                bssCOMRAM                            61       61        8        1       1
                cinit                              1CEE     1CEE       64      305       0
                nvCOMRAM                             69       69        3        1       1
                idataCOMRAM                        1F6C     1F6C        3      305       0

TOTAL           Name                               Link     Load   Length     Space
        CLASS   CODE           
                intcode                               8        8       AA         0
                text                               1F70     1F70        2         0
                init                                 B2       B2        4         0
                reset_vec                             0        0        6         0
                text31                             1DA2     1DA2       48         0
                text29                             1DEA     1DEA       34         0
                text28                             1F14     1F14        C         0
                text27                             1F08     1F08        C         0
                text26                             1E1E     1E1E       26         0
                text25                             1EA4     1EA4       1E         0
                text24                             1E44     1E44       24         0
                text23                             1E86     1E86       1E         0
                text22                             1A4C     1A4C       FA         0
                text21                             1C0C     1C0C       7C         0
                text20                             1E68     1E68       1E         0
                text19                             1C88     1C88       66         0
                text18                             1F52     1F52        A         0
                text17                             1F48     1F48        A         0
                text16                             1F3E     1F3E        A         0
                text15                             1F34     1F34        A         0
                text14                             1EDE     1EDE       1A         0
                text13                              60A      60A      5A8         0
                text12                             1056     1056      432         0
                text11                              BB2      BB2      4A4         0
                text10                             1916     1916      136         0
                text9                              1B46     1B46       C6         0
                text8                              1EF8     1EF8       10         0
                text7                              1F64     1F64        8         0
                text6                              1F5C     1F5C        8         0
                text5                              1EC2     1EC2       1C         0
                text4                              1D52     1D52       50         0
                text3                              1488     1488      358         0
                text2                              1F2A     1F2A        A         0
                text1                              1F20     1F20        A         0
                text0                              17E0     17E0      136         0
                cinit                              1CEE     1CEE       64         0
                idataCOMRAM                        1F6C     1F6C        3         0

        CLASS   CONST          

        CLASS   SMALLCONST     
                smallconst                          600      600        A         0

        CLASS   MEDIUMCONST    

        CLASS   COMRAM         
                temp                                 6F       6F        1         1
                cstackCOMRAM                          1        1       60         1
                dataCOMRAM                           6C       6C        3         1
                bssCOMRAM                            61       61        8         1
                nvCOMRAM                             69       69        3         1

        CLASS   ABS1           

        CLASS   BIGRAM         

        CLASS   RAM            

        CLASS   BANK0          
                cstackBANK0                          AA       AA       1A         1
                bssBANK0                             80       80       2A         1

        CLASS   BANK1          
                bssBANK1                            100      100       64         1

        CLASS   BANK2          
                bssBANK2                            200      200       FF         1

        CLASS   BANK3          

        CLASS   BANK4          

        CLASS   BANK5          

        CLASS   SFR            

        CLASS   BIGSFR         

        CLASS   CONFIG         
                config                           300000   300000        E         4

        CLASS   IDLOC          
                idloc                            200000   200000        8         5

        CLASS   EEDATA         

        CLASS   FARRAM         

        CLASS   HEAP           

        CLASS   STACK          



SEGMENTS        Name                           Load    Length   Top    Selector   Space  Class

                bssBANK2                       000200  0000FF  0002FF       200       1  BANK2   
                bssBANK1                       000100  000064  000164       100       1  BANK1   
                bssBANK0                       000080  000044  0000C4        80       1  BANK0   
                text13                         00060A  001965  001F6F       305       0  CODE    
                text                           001F70  000002  001F72       FB8       0  CODE    
                cstackCOMRAM                   000001  00006F  000070         1       1  COMRAM  
                reset_vec                      000000  000006  000006         0       0  CODE    
                intcode                        000008  0000AE  0000B6         4       0  CODE    
                smallconst                     000600  00000A  00060A       300       0  SMALLCON


UNUSED ADDRESS RANGES

        Name                Unused          Largest block    Delta
        BANK0            0000C4-0000FF               3C
        BANK1            000164-0001FF               9C
        BANK2            0002FF-0002FF                1
        BANK3            000300-0003FF              100
        BANK4            000400-0004FF              100
        BANK5            000500-0005FF              100
        BIGRAM           000070-00007F               10
                         0000C4-0000FF               3C
                         000164-0001FF               9C
                         0002FF-0005FF              301
        BIGSFR           000F80-000FFF               80
        CODE             000006-000007                2
                         0000B6-0005FF              54A
                         001F6F-001F6F                1
                         001F72-007FFF             208E
        COMRAM           000070-00007F               10
        CONST            000006-000007                2
                         0000B6-0005FF              54A
                         001F6F-001F6F                1
                         001F72-007FFF             608E
        EEDATA           F00000-F000FF              100
        MEDIUMCONST      001F6F-001F6F                1
                         001F72-007FFF             608E
        RAM              0000C4-0000FF               3C
                         000164-0001FF               9C
                         0002FF-0005FF              100
        SFR              000F80-000FFF               80
        SMALLCONST       001F6F-001F6F                1
                         001F72-007FFF              100

                                  Symbol Table

?___fladd                                                                      cstackCOMRAM 000041
?___fldiv                                                                      cstackCOMRAM 00000F
?___flmul                                                                      cstackCOMRAM 000028
?___fltol                                                                      cstackCOMRAM 000051
I2C_Master_Write@data                                                          cstackCOMRAM 000010
IO_Expander_Write@Data                                                         cstackCOMRAM 000011
LCD_CMD@CMD                                                                    cstackCOMRAM 000013
LCD_Init@I2C_Add                                                               cstackCOMRAM 000016
LCD_Set_Cursor@COL                                                             cstackCOMRAM 000014
LCD_Set_Cursor@ROW                                                             cstackCOMRAM 000017
LCD_Write_4Bit@Nibble                                                          cstackCOMRAM 000012
LCD_Write_Char@Data                                                            cstackCOMRAM 000013
LCD_Write_String@Str                                                           cstackCOMRAM 000014
LCD_Write_String@i                                                             cstackCOMRAM 000018
_ACKDT                                                                         (abs)        007E2D
_ACKEN                                                                         (abs)        007E2C
_ACKSTAT                                                                       (abs)        007E2E
_ADCON1                                                                        (abs)        000FC1
_BackLight_State                                                               dataCOMRAM   00006E
_CCP1CON                                                                       (abs)        000FBD
_CCP2CON                                                                       (abs)        000FBA
_CCPR1L                                                                        (abs)        000FBE
_CCPR2L                                                                        (abs)        000FBB
_I2C_Master_Init                                                               text14       001EDE
_I2C_Master_Start                                                              text28       001F14
_I2C_Master_Stop                                                               text27       001F08
_I2C_Master_Wait                                                               text29       001DEA
_I2C_Master_Write                                                              text26       001E1E
_INTCONbits                                                                    (abs)        000FF2
_IO_Expander_Write                                                             text25       001EA4
_LATAbits                                                                      (abs)        000F89
_LCD_CMD                                                                       text23       001E86
_LCD_Init                                                                      text22       001A4C
_LCD_Set_Cursor                                                                text21       001C0C
_LCD_Write_4Bit                                                                text24       001E44
_LCD_Write_Char                                                                text20       001E68
_LCD_Write_String                                                              text19       001C88
_PEN                                                                           (abs)        007E2A
_PIE1bits                                                                      (abs)        000F9D
_PIR1bits                                                                      (abs)        000F9E
_PR2                                                                           (abs)        000FCB
_RCEN                                                                          (abs)        007E2B
_RCONbits                                                                      (abs)        000FD0
_RCREG                                                                         (abs)        000FAE
_RCSTAbits                                                                     (abs)        000FAB
_RS                                                                            bssCOMRAM    000068
_RSEN                                                                          (abs)        007E29
_SEN                                                                           (abs)        007E28
_SPBRG                                                                         (abs)        000FAF
_SSPADD                                                                        (abs)        000FC8
_SSPBUF                                                                        (abs)        000FC9
_SSPCON1                                                                       (abs)        000FC6
_SSPCON2                                                                       (abs)        000FC5
_SSPIF                                                                         (abs)        007CF3
_SSPSTAT                                                                       (abs)        000FC7
_T2CON                                                                         (abs)        000FCA
_TRISA                                                                         (abs)        000F92
_TRISBbits                                                                     (abs)        000F93
_TRISC3                                                                        (abs)        007CA3
_TRISC4                                                                        (abs)        007CA4
_TRISC6                                                                        (abs)        007CA6
_TRISC7                                                                        (abs)        007CA7
_TRISCbits                                                                     (abs)        000F94
_TXREG                                                                         (abs)        000FAD
_TXSTAbits                                                                     (abs)        000FAC
__HRAM                                                                         (abs)        000000
__Habs1                                                                        abs1         000000
__Hbank0                                                                       bank0        000000
__Hbank1                                                                       bank1        000000
__Hbank2                                                                       bank2        000000
__Hbank3                                                                       bank3        000000
__Hbank4                                                                       bank4        000000
__Hbank5                                                                       bank5        000000
__Hbigbss                                                                      bigbss       000000
__Hbigdata                                                                     bigdata      000000
__Hbigram                                                                      bigram       000000
__Hbigsfr                                                                      bigsfr       000000
__Hbss                                                                         bss          000000
__HbssBANK0                                                                    bssBANK0     000000
__HbssBANK1                                                                    bssBANK1     000000
__HbssBANK2                                                                    bssBANK2     000000
__HbssCOMRAM                                                                   bssCOMRAM    000000
__Hcinit                                                                       cinit        000000
__Hclrtext                                                                     clrtext      000000
__Hcomram                                                                      comram       000000
__Hconfig                                                                      config       30000E
__Hconst                                                                       const        000000
__HcstackBANK0                                                                 cstackBANK0  000000
__HcstackCOMRAM                                                                cstackCOMRAM 000000
__Hdata                                                                        data         000000
__HdataCOMRAM                                                                  dataCOMRAM   000000
__Heeprom_data                                                                 eeprom_data  000000
__Hfarbss                                                                      farbss       000000
__Hfardata                                                                     fardata      000000
__Hheap                                                                        heap         000000
__Hibigdata                                                                    ibigdata     000000
__Hidata                                                                       idata        000000
__HidataCOMRAM                                                                 idataCOMRAM  000000
__Hidloc                                                                       idloc        200008
__Hifardata                                                                    ifardata     000000
__Hinit                                                                        init         0000B6
__Hintcode                                                                     intcode      0000B2
__Hintcode_body                                                                intcode_body 000000
__Hintcodelo                                                                   intcodelo    0000B2
__Hintentry                                                                    intentry     000000
__Hintret                                                                      intret       000000
__Hintsave_regs                                                                intsave_regs 000000
__Hirdata                                                                      irdata       000000
__Hmediumconst                                                                 mediumconst  000000
__HnvCOMRAM                                                                    nvCOMRAM     000000
__HnvFARRAM                                                                    nvFARRAM     000000
__Hnvbit                                                                       nvbit        000000
__Hnvrram                                                                      nvrram       000000
__Hparam                                                                       rparam       000000
__Hpowerup                                                                     powerup      0000B2
__Hram                                                                         ram          000000
__Hramtop                                                                      ramtop       000600
__Hrbit                                                                        rbit         000000
__Hrbss                                                                        rbss         000000
__Hrdata                                                                       rdata        000000
__Hreset_vec                                                                   reset_vec    000006
__Hrparam                                                                      rparam       000000
__Hsfr                                                                         sfr          000000
__Hsmallconst                                                                  smallconst   00060A
__Hspace_0                                                                     (abs)        001F72
__Hspace_1                                                                     (abs)        0002FF
__Hspace_2                                                                     (abs)        000000
__Hspace_4                                                                     (abs)        60000E
__Hstack                                                                       stack        000000
__Hstruct                                                                      struct       000000
__Htemp                                                                        temp         000070
__Htext                                                                        text         000000
__Htext0                                                                       text0        000000
__Htext1                                                                       text1        000000
__Htext10                                                                      text10       000000
__Htext11                                                                      text11       000000
__Htext12                                                                      text12       000000
__Htext13                                                                      text13       000000
__Htext14                                                                      text14       000000
__Htext15                                                                      text15       000000
__Htext16                                                                      text16       000000
__Htext17                                                                      text17       000000
__Htext18                                                                      text18       000000
__Htext19                                                                      text19       000000
__Htext2                                                                       text2        000000
__Htext20                                                                      text20       000000
__Htext21                                                                      text21       000000
__Htext22                                                                      text22       000000
__Htext23                                                                      text23       000000
__Htext24                                                                      text24       000000
__Htext25                                                                      text25       000000
__Htext26                                                                      text26       000000
__Htext27                                                                      text27       000000
__Htext28                                                                      text28       000000
__Htext29                                                                      text29       000000
__Htext3                                                                       text3        000000
__Htext31                                                                      text31       000000
__Htext4                                                                       text4        000000
__Htext5                                                                       text5        000000
__Htext6                                                                       text6        000000
__Htext7                                                                       text7        000000
__Htext8                                                                       text8        000000
__Htext9                                                                       text9        000000
__LRAM                                                                         (abs)        000001
__Labs1                                                                        abs1         000000
__Lbank0                                                                       bank0        000000
__Lbank1                                                                       bank1        000000
__Lbank2                                                                       bank2        000000
__Lbank3                                                                       bank3        000000
__Lbank4                                                                       bank4        000000
__Lbank5                                                                       bank5        000000
__Lbigbss                                                                      bigbss       000000
__Lbigdata                                                                     bigdata      000000
__Lbigram                                                                      bigram       000000
__Lbigsfr                                                                      bigsfr       000000
__Lbss                                                                         bss          000000
__LbssBANK0                                                                    bssBANK0     000000
__LbssBANK1                                                                    bssBANK1     000000
__LbssBANK2                                                                    bssBANK2     000000
__LbssCOMRAM                                                                   bssCOMRAM    000000
__Lcinit                                                                       cinit        000000
__Lclrtext                                                                     clrtext      000000
__Lcomram                                                                      comram       000000
__Lconfig                                                                      config       000000
__Lconst                                                                       const        000000
__LcstackBANK0                                                                 cstackBANK0  000000
__LcstackCOMRAM                                                                cstackCOMRAM 000000
__Ldata                                                                        data         000000
__LdataCOMRAM                                                                  dataCOMRAM   000000
__Leeprom_data                                                                 eeprom_data  000000
__Lfarbss                                                                      farbss       000000
__Lfardata                                                                     fardata      000000
__Lheap                                                                        heap         000000
__Libigdata                                                                    ibigdata     000000
__Lidata                                                                       idata        000000
__LidataCOMRAM                                                                 idataCOMRAM  000000
__Lidloc                                                                       idloc        000000
__Lifardata                                                                    ifardata     000000
__Linit                                                                        init         0000B2
__Lintcode                                                                     intcode      000008
__Lintcode_body                                                                intcode_body 000000
__Lintcodelo                                                                   intcodelo    0000B2
__Lintentry                                                                    intentry     000000
__Lintret                                                                      intret       000000
__Lintsave_regs                                                                intsave_regs 000000
__Lirdata                                                                      irdata       000000
__Lmediumconst                                                                 mediumconst  000000
__LnvCOMRAM                                                                    nvCOMRAM     000000
__LnvFARRAM                                                                    nvFARRAM     000000
__Lnvbit                                                                       nvbit        000000
__Lnvrram                                                                      nvrram       000000
__Lparam                                                                       rparam       000000
__Lpowerup                                                                     powerup      0000B2
__Lram                                                                         ram          000000
__Lramtop                                                                      ramtop       000600
__Lrbit                                                                        rbit         000000
__Lrbss                                                                        rbss         000000
__Lrdata                                                                       rdata        000000
__Lreset_vec                                                                   reset_vec    000000
__Lrparam                                                                      rparam       000000
__Lsfr                                                                         sfr          000000
__Lsmallconst                                                                  smallconst   000600
__Lspace_0                                                                     (abs)        000000
__Lspace_1                                                                     (abs)        000000
__Lspace_2                                                                     (abs)        000000
__Lspace_4                                                                     (abs)        000000
__Lstack                                                                       stack        000000
__Lstruct                                                                      struct       000000
__Ltemp                                                                        temp         00006F
__Ltext                                                                        text         000000
__Ltext0                                                                       text0        000000
__Ltext1                                                                       text1        000000
__Ltext10                                                                      text10       000000
__Ltext11                                                                      text11       000000
__Ltext12                                                                      text12       000000
__Ltext13                                                                      text13       000000
__Ltext14                                                                      text14       000000
__Ltext15                                                                      text15       000000
__Ltext16                                                                      text16       000000
__Ltext17                                                                      text17       000000
__Ltext18                                                                      text18       000000
__Ltext19                                                                      text19       000000
__Ltext2                                                                       text2        000000
__Ltext20                                                                      text20       000000
__Ltext21                                                                      text21       000000
__Ltext22                                                                      text22       000000
__Ltext23                                                                      text23       000000
__Ltext24                                                                      text24       000000
__Ltext25                                                                      text25       000000
__Ltext26                                                                      text26       000000
__Ltext27                                                                      text27       000000
__Ltext28                                                                      text28       000000
__Ltext29                                                                      text29       000000
__Ltext3                                                                       text3        000000
__Ltext31                                                                      text31       000000
__Ltext4                                                                       text4        000000
__Ltext5                                                                       text5        000000
__Ltext6                                                                       text6        000000
__Ltext7                                                                       text7        000000
__Ltext8                                                                       text8        000000
__Ltext9                                                                       text9        000000
__S0                                                                           (abs)        001F72
__S1                                                                           (abs)        0002FF
__S4                                                                           (abs)        000000
__S5                                                                           (abs)        000000
___fladd                                                                       text13       00060A
___fladd@a                                                                     cstackCOMRAM 000045
___fladd@aexp                                                                  cstackCOMRAM 00004E
___fladd@b                                                                     cstackCOMRAM 000041
___fladd@bexp                                                                  cstackCOMRAM 00004F
___fladd@grs                                                                   cstackCOMRAM 000050
___fladd@signs                                                                 cstackCOMRAM 00004D
___fldiv                                                                       text12       001056
___fldiv@a                                                                     cstackCOMRAM 000013
___fldiv@aexp                                                                  cstackCOMRAM 000027
___fldiv@b                                                                     cstackCOMRAM 00000F
___fldiv@bexp                                                                  cstackCOMRAM 000026
___fldiv@grs                                                                   cstackCOMRAM 000022
___fldiv@new_exp                                                               cstackCOMRAM 000020
___fldiv@rem                                                                   cstackCOMRAM 00001B
___fldiv@sign                                                                  cstackCOMRAM 00001F
___flmul                                                                       text11       000BB2
___flmul@a                                                                     cstackCOMRAM 00002C
___flmul@aexp                                                                  cstackCOMRAM 000039
___flmul@b                                                                     cstackCOMRAM 000028
___flmul@bexp                                                                  cstackCOMRAM 00003A
___flmul@grs                                                                   cstackCOMRAM 000035
___flmul@prod                                                                  cstackCOMRAM 00003B
___flmul@sign                                                                  cstackCOMRAM 000034
___flmul@temp                                                                  cstackCOMRAM 00003F
___fltol                                                                       text10       001916
___fltol@exp1                                                                  cstackCOMRAM 00005A
___fltol@f1                                                                    cstackCOMRAM 000051
___fltol@sign1                                                                 cstackCOMRAM 000059
___heap_hi                                                                     (abs)        000000
___heap_lo                                                                     (abs)        000000
___inthi_sp                                                                    stack        000000
___intlo_sp                                                                    stack        000000
___param_bank                                                                  (abs)        000000
___rparam_used                                                                 (abs)        000001
___sp                                                                          stack        000000
__accesstop                                                                    (abs)        000080
__activetblptr                                                                 (abs)        000002
__cntErrataNOP_/tmp/xcXMhfnii.o                                                (abs)        000001
__cntErrataNOP_dist/default/production/UART_TX_18F452_2.X__copia_.production.o (abs)        000164
__end_of_I2C_Master_Init                                                       text14       001EF8
__end_of_I2C_Master_Start                                                      text28       001F20
__end_of_I2C_Master_Stop                                                       text27       001F14
__end_of_I2C_Master_Wait                                                       text29       001E1E
__end_of_I2C_Master_Write                                                      text26       001E44
__end_of_IO_Expander_Write                                                     text25       001EC2
__end_of_LCD_CMD                                                               text23       001EA4
__end_of_LCD_Init                                                              text22       001B46
__end_of_LCD_Set_Cursor                                                        text21       001C88
__end_of_LCD_Write_4Bit                                                        text24       001E68
__end_of_LCD_Write_Char                                                        text20       001E86
__end_of_LCD_Write_String                                                      text19       001CEE
__end_of___fladd                                                               text13       000BB2
__end_of___fldiv                                                               text12       001488
__end_of___flmul                                                               text11       001056
__end_of___fltol                                                               text10       001A4C
__end_of__initialization                                                       cinit        001D44
__end_of_adelanteL                                                             text18       001F5C
__end_of_adelanteR                                                             text17       001F52
__end_of_adint                                                                 intcode      0000B2
__end_of_atrasL                                                                text16       001F48
__end_of_atrasR                                                                text15       001F3E
__end_of_boot                                                                  text4        001DA2
__end_of_globalPWM                                                             text9        001C0C
__end_of_init_interrupts                                                       text8        001F08
__end_of_init_uart                                                             text5        001EDE
__end_of_main                                                                  text0        001916
__end_of_rx_start                                                              text7        001F6C
__end_of_setPWM                                                                text3        0017E0
__end_of_stopL                                                                 text2        001F34
__end_of_stopR                                                                 text1        001F2A
__end_of_strcpy                                                                text31       001DEA
__end_of_tx_start                                                              text6        001F64
__initialization                                                               cinit        001CEE
__mediumconst                                                                  mediumconst  000000
__pbssBANK0                                                                    bssBANK0     000080
__pbssBANK1                                                                    bssBANK1     000100
__pbssBANK2                                                                    bssBANK2     000200
__pbssCOMRAM                                                                   bssCOMRAM    000061
__pcinit                                                                       cinit        001CEE
__pcstackBANK0                                                                 cstackBANK0  0000AA
__pcstackCOMRAM                                                                cstackCOMRAM 000001
__pdataCOMRAM                                                                  dataCOMRAM   00006C
__pidataCOMRAM                                                                 idataCOMRAM  001F6C
__pintcode                                                                     intcode      000008
__pnvCOMRAM                                                                    nvCOMRAM     000069
__psmallconst                                                                  smallconst   000600
__ptext0                                                                       text0        0017E0
__ptext1                                                                       text1        001F20
__ptext10                                                                      text10       001916
__ptext11                                                                      text11       000BB2
__ptext12                                                                      text12       001056
__ptext13                                                                      text13       00060A
__ptext14                                                                      text14       001EDE
__ptext15                                                                      text15       001F34
__ptext16                                                                      text16       001F3E
__ptext17                                                                      text17       001F48
__ptext18                                                                      text18       001F52
__ptext19                                                                      text19       001C88
__ptext2                                                                       text2        001F2A
__ptext20                                                                      text20       001E68
__ptext21                                                                      text21       001C0C
__ptext22                                                                      text22       001A4C
__ptext23                                                                      text23       001E86
__ptext24                                                                      text24       001E44
__ptext25                                                                      text25       001EA4
__ptext26                                                                      text26       001E1E
__ptext27                                                                      text27       001F08
__ptext28                                                                      text28       001F14
__ptext29                                                                      text29       001DEA
__ptext3                                                                       text3        001488
__ptext31                                                                      text31       001DA2
__ptext4                                                                       text4        001D52
__ptext5                                                                       text5        001EC2
__ptext6                                                                       text6        001F5C
__ptext7                                                                       text7        001F64
__ptext8                                                                       text8        001EF8
__ptext9                                                                       text9        001B46
__ramtop                                                                       ramtop       000600
__smallconst                                                                   smallconst   000600
_adelanteL                                                                     text18       001F52
_adelanteR                                                                     text17       001F48
_adint                                                                         intcode      000008
_atrasL                                                                        text16       001F3E
_atrasR                                                                        text15       001F34
_boot                                                                          text4        001D52
_cont_rc                                                                       bssCOMRAM    000063
_data                                                                          bssCOMRAM    000067
_duty_temp                                                                     bssCOMRAM    000061
_frec_osc                                                                      bssBANK0     0000A2
_globalPWM                                                                     text9        001B46
_globalPWM$1409                                                                cstackCOMRAM 00005B
_i2c_add                                                                       nvCOMRAM     00006B
_init_interrupts                                                               text8        001EF8
_init_uart                                                                     text5        001EC2
_main                                                                          text0        0017E0
_mask                                                                          dataCOMRAM   00006C
_periodo                                                                       nvCOMRAM     000069
_pwm_p                                                                         bssBANK0     0000A6
_rc_buff                                                                       bssBANK1     000100
_rc_data                                                                       bssBANK2     000200
_rx_start                                                                      text7        001F64
_setPWM                                                                        text3        001488
_setPWM$1410                                                                   cstackBANK0  0000BC
_setPWM$1411                                                                   cstackBANK0  0000C0
_stopL                                                                         text2        001F2A
_stopR                                                                         text1        001F20
_strcpy                                                                        text31       001DA2
_test_buff                                                                     bssBANK0     000080
_tmr2_presc                                                                    bssBANK0     00009E
_tx_start                                                                      text6        001F5C
_valor_prueba_debug                                                            bssCOMRAM    000066
_valor_prueba_debug2                                                           bssCOMRAM    000065
btemp                                                                          temp         00006F
end_of_initialization                                                          cinit        001D44
globalPWM@freq_osc                                                             cstackBANK0  0000AE
globalPWM@period_pwm                                                           cstackBANK0  0000AA
globalPWM@presc                                                                cstackBANK0  0000B2
int$flags                                                                      temp         00006F
intlevel0                                                                      text         001F70
intlevel1                                                                      text         001F70
intlevel2                                                                      text         001F70
intlevel3                                                                      text         001F70
isa$std                                                                        (abs)        000001
isa$xinst                                                                      (abs)        000000
setPWM@freq_osc                                                                cstackBANK0  0000B2
setPWM@module                                                                  cstackBANK0  0000BA
setPWM@period_pwm                                                              cstackBANK0  0000AA
setPWM@presc                                                                   cstackBANK0  0000B6
setPWM@pwm_duty                                                                cstackBANK0  0000AE
stackhi                                                                        (abs)        000000
stacklo                                                                        (abs)        000000
start                                                                          init         0000B2
start_initialization                                                           cinit        001CEE
strcpy@d                                                                       cstackCOMRAM 000007
strcpy@dest                                                                    cstackCOMRAM 000001
strcpy@s                                                                       cstackCOMRAM 000005
strcpy@src                                                                     cstackCOMRAM 000003
ttemp5                                                                         temp         000070
ttemp6                                                                         temp         000073
ttemp7                                                                         temp         000077
wtemp8                                                                         temp         000070


MODULE INFORMATION

Module		Function		Class		Link	Load	Size
lcd_i2c.c
		_LCD_Init      		CODE           	1A4C	0000	250
		_LCD_Write_4Bit		CODE           	1E44	0000	36
		_LCD_Write_Char		CODE           	1E68	0000	30
		_LCD_CMD       		CODE           	1E86	0000	30
		_I2C_Master_Wait		CODE           	1DEA	0000	52
		_I2C_Master_Init		CODE           	1EDE	0000	26
		_I2C_Master_Stop		CODE           	1F08	0000	12
		_LCD_Set_Cursor		CODE           	1C0C	0000	124
		_IO_Expander_Write		CODE           	1EA4	0000	30
		_I2C_Master_Write		CODE           	1E1E	0000	38
		_I2C_Master_Start		CODE           	1F14	0000	12
		_LCD_Write_String		CODE           	1C88	0000	102

lcd_i2c.c estimated size: 742

mainTx.c
		_adint         		CODE           	0008	0000	170
		_adelanteL     		CODE           	1F52	0000	10
		_adelanteR     		CODE           	1F48	0000	10
		_boot          		CODE           	1D52	0000	80
		_stopL         		CODE           	1F2A	0000	10
		_main          		CODE           	17E0	0000	310
		_stopR         		CODE           	1F20	0000	10
		_init_uart     		CODE           	1EC2	0000	28
		_globalPWM     		CODE           	1B46	0000	198
		_rx_start      		CODE           	1F64	0000	8
		_tx_start      		CODE           	1F5C	0000	8
		_atrasL        		CODE           	1F3E	0000	10
		_setPWM        		CODE           	1488	0000	856
		_init_interrupts		CODE           	1EF8	0000	16
		_atrasR        		CODE           	1F34	0000	10

mainTx.c estimated size: 1734

/opt/microchip/xc8/v2.36/pic/sources/c99/common/sprcmul.c
		___flmul       		CODE           	0BB2	0000	1188

/opt/microchip/xc8/v2.36/pic/sources/c99/common/sprcmul.c estimated size: 1188

/opt/microchip/xc8/v2.36/pic/sources/c99/common/sprcdiv.c
		___fldiv       		CODE           	1056	0000	1074

/opt/microchip/xc8/v2.36/pic/sources/c99/common/sprcdiv.c estimated size: 1074

shared
		__initialization		CODE           	1CEE	0000	86

shared estimated size: 86

/opt/microchip/xc8/v2.36/pic/sources/c99/common/strcpy.c
		_strcpy        		CODE           	1DA2	0000	72

/opt/microchip/xc8/v2.36/pic/sources/c99/common/strcpy.c estimated size: 72

/opt/microchip/xc8/v2.36/pic/sources/c99/common/fltol.c
		___fltol       		CODE           	1916	0000	310

/opt/microchip/xc8/v2.36/pic/sources/c99/common/fltol.c estimated size: 310

/opt/microchip/xc8/v2.36/pic/sources/c99/common/sprcadd.c
		___fladd       		CODE           	060A	0000	1448

/opt/microchip/xc8/v2.36/pic/sources/c99/common/sprcadd.c estimated size: 1448

